:0400000002011F32A8
:03000B0002007080
:03017D0002000E6F
:05000E0012001F80FE3E
:0A001300907F9C74FFF01200CA02F7
:02001D00005190
:05001F00120013D2AF36
:040024007A207B4E75
:050028001ABAFF011BE4
:04002D00EA4B70F733
:0500310012010D80EE3C
:0100360022A7
:05017800E4F50AF50B9F
:0C003700AA087B00EA258AF58AAA097B4A
:0600430000EA258CF58C9B
:010049002294
:06004A0085820885830990
:01005000228D
:0E005100C28C538EF753890F438901758A00C4
:0E005F00758C0090B1E012004A120037D2A951
:02006D00D28C33
:01006F00226E
:0E007000C0E0C0F0C082C083C002C003C00464
:0E007E00C005C006C007C000C001C0D075D0CC
:0C008C0000C28C120037D28C050AE4B5CB
:040098000A02050B48
:09009C00E50AB40A04E50B600258
:0200A5008008D1
:0700A7001200EDE4F50AF57B
:0100AE000B46
:0E00AF00D0D0D001D000D007D006D005D004AC
:0D00BD00D003D002D083D082D0F0D0E0324A
:0E00CA00907F93E0FA54CFF0907F9CE0FA44D0
:0200D80030F006
:0100DA002203
:0800DB00907F96E0FA4410F05A
:0100E30022FA
:0800E400907F96E0FA54EFF062
:0100EC0022F1
:0800ED00907F96E0FA30E40375
:0300F5000200E422
:0300F8000200DB28
:0800FB00907F96E0FA4420F02A
:0101030022D9
:08010400907F96E0FA54DFF051
:01010C0022D0
:08010D00907F96E0FA30E50353
:03011500020104E0
:030118000200FBE7
:06014E00E478FFF6D8FD85
:08012C007900E94400601B7A30
:0501340000900180783D
:030139000075A0AE
:0C013C0000E493F2A308B8000205A0D96B
:06014800F4DAF275A0FFDD
:080154007800E84400600A791C
:03015C000075A08B
:06015F0000E4F309D8FCE6
:080165007800E84400600C7909
:0B016D0000900000E4F0A3D8FCD9FAD9
:03011F0075810BDC
:0A01220012011BE582600302000ECB
:03011B00758200EA
:01011E0022BE
:00000001FF
